:100000000C943B000C9458000C945A000C9458002B
:100010000C9458000C9458000C9458000C94580000
:100020000C9458000C9458000C9458000C945800F0
:100030000C9458000C94B7000C9458000C94580081
:100040000C9458000C9458000C9458000C945800D0
:100050000C9458000C9458000C9458000C945800C0
:100060000C9458000C945800AA02AE02B202B502D9
:10007000B902BD02AA0211241FBECFEFD8E0DEBF35
:10008000CDBF11E0A0E0B1E0E0E6FDE002C00590E8
:100090000D92AA30B107D9F721E0AAE0B1E001C082
:1000A0001D92AA31B207E1F70E9408030C94AE0634
:1000B0000C9400001F920F920FB60F9211242F93F1
:1000C0003F938F939F93AF93BF93EF93FF93E998E1
:1000D0008091160190911701A0911801B09119011A
:1000E000E4E8F0E020813181820F931FA11DB11D52
:1000F0008093120190931301A0931401B093150102
:100100008091120190911301A0911401B0911501F9
:10011000B695A7959795879580930A0190930B01C3
:10012000A0930C01B0930D01118210821092160160
:1001300010921701109218011092190110920E01DD
:1001400010920F01109210011092110198B182E0EB
:10015000892788B9FF91EF91BF91AF919F918F91BE
:100160003F912F910F900FBE0F901F9018951F92E7
:100170000F920FB60F9211248F939F93AF93BF935B
:100180008091160190911701A0911801B091190169
:1001900011968093160190931701A0931801B093C4
:1001A0001901BF91AF919F918F910F900FBE0F904A
:1001B0001F901895409A00C000C000C0409800C031
:1001C00000C000C000C000C000C000C00000089512
:1001D000409A00C000C000C000C000C000C000C005
:1001E000409800C000C000C000C00895AF92BF9208
:1001F000CF92DF92EF92FF920F931F93CF93DF93F3
:10020000C82EE42EC8E0D0E000E810E0A62EB12C05
:10021000C8018A219B21892B19F00E94E80002C0A5
:100220000E94DA0015950795219791F7C8E0D0E074
:1002300000E810E0D12CC8018C219D21892B19F0F8
:100240000E94E80002C00E94DA00159507952197E8
:1002500091F7C8E0D0E000E810E0F12CC8018E2151
:100260009F21892B19F00E94E80002C00E94DA0049
:1002700015950795219791F7DF91CF911F910F91D8
:10028000FF90EF90DF90CF90BF90AF9008952F92A6
:100290003F924F925F926F927F928F929F92AF9216
:1002A000BF92CF92DF92EF92FF920F931F93CF9363
:1002B000DF93CDB7DEB72A970FB6F894DEBF0FBE37
:1002C000CDBFD82EC92EF7010130110501F13B0138
:1002D0002901461A570A842F90E0BC016D19710953
:1002E0007E836D83852F90E09C012C19310938871E
:1002F0002F8333961A861986E12CF12C80E090E04A
:1003000020E030E0580141E0A41AB10805C0608344
:100310007183828393833DC01C01240C351C4D8165
:100320005E814E0D5F1D5A8349834F8158856985D3
:100330007A85460F571F5C834B832017310749F19D
:100340004F0153E0851A9108B5010E948006660DA1
:10035000771DD4016D937C934F01B1E08B1A910806
:10036000C701B5010E9480066D0DD4016C9389858B
:100370009A85B5010E9480066C0D60832F5F3F4F08
:1003800034964B815C815A874987E980FA80C101A4
:10039000C3CF2A960FB6F894DEBF0FBECDBFDF9154
:1003A000CF911F910F91FF90EF90DF90CF90BF9072
:1003B000AF909F908F907F906F905F904F903F9005
:1003C0002F9008952F923F924F925F926F927F925B
:1003D0008F929F92AF92BF92CF92DF92EF92FF9255
:1003E0000F931F93CF93DF9300D000D0CDB7DEB72C
:1003F000FC01B2803380B11004C0232C3B823C82CC
:10040000C2C0FC0100811181B8010836F1E01F076C
:1004100010F06856714080E090E00E9485052B0145
:100420003C01632D70E080E090E00E94850520E0B3
:1004300030E048EC52E40E94E4046B017C016B2D37
:1004400070E080E090E00E94850520E030E048EC1C
:1004500052E40E94E4044B015C0120E030E040E7FC
:1004600052E4C301B2010E94E4042B013C010E944A
:1004700056056A8370E080E090E00E9487059B014A
:10048000AC01C301B2010E9477042B013C01A5011C
:10049000940160E070E080E89FE30E9477049B0194
:1004A000AC01C701B6010E94130620E030E040E035
:1004B00053E40E9413060E945605262EA3019201C2
:1004C000C501B4010E9413069B01AC0160E070E01D
:1004D00080E89FE30E9477049B01AC01C701B6014D
:1004E0000E94130620E030E040E053E40E9413062F
:1004F0000E9456056983A301920160E070E080E8E4
:100500009FE30E9477049B01AC01C501B4010E94E6
:1005100013069B01AC0160E070E080E89FE30E945D
:1005200077049B01AC01C701B6010E94130620E0CD
:1005300030E040E053E40E9413060E9456052A81F1
:10054000822F90E087309105E8F4FC01EC5CFF4FCE
:100550000C9494062B826C83232C15C02B823C8236
:10056000298011C06B833C820EC03B8289818C83C1
:100570000AC03B822C82262E06C0E981EB832C82A6
:10058000202E01C0212C622D7C818B810F900F9039
:100590000F900F90DF91CF911F910F91FF90EF90EF
:1005A000DF90CF90BF90AF909F908F907F906F9093
:1005B0005F904F903F902F900895CF92DF92EF92EF
:1005C000FF920F931F93CF93DF936A01EB017C019E
:1005D00000E010E00C151D0561F0C7010E94E2016A
:1005E0006993799389930F5F1F4F84E0E80EF11CA4
:1005F000F1CFDF91CF911F910F91FF90EF90DF909E
:10060000CF900895282F862F622F792F942F089549
:10061000CF93DF93CDB7DEB7C25DD1090FB6F894A3
:10062000DEBF0FBECDBFE99A809169008C608093D8
:10063000690080916F00816080936F0080918100DC
:100640008160809381008FB780688FBF8FE387B907
:1006500018B8809100019091010144E164E60E9484
:1006600002034B015C01809102019091030144E17E
:1006700064E60E9402039E012F5F3F4F79010EE165
:1006800010E0A50194010E9447014EE150E0BE0137
:1006900067587F4FC7010E94DD0249E7A42EB12CA5
:1006A000AC0EBD1E32E0A30EB11C4E0185ED880ECE
:1006B000911C8501D8011197C8010297F80140816A
:1006C0006C91FC0180810E94F6000D5F1F4F0815A0
:1006D000190581F78091020190910301089690938A
:1006E000030180930201809100019091010108971C
:1006F000909301018093000180910001909101018C
:1007000044E164E60E9402032B013C018091020156
:100710009091030144E164E60E9402039E012F5F71
:100720003F4F79010EE110E0A30192010E944701C1
:100730004EE150E0BE0167587F4FC7010E94DD02C5
:10074000DD24D39434E0C32E40911601509117015B
:100750006091180170911901809184009091850039
:10076000480F591F611D711D80910A0190910B0165
:10077000A0910C01B0910D0184179507A607B7074A
:1007800008F4E99A8091120190911301A09114014B
:10079000B091150125E0B695A795979587952A956F
:1007A000D1F700910E0110910F01209110013091AD
:1007B0001101080F191F2A1F3B1F041715072607D1
:1007C000370710F640910E0150910F016091100112
:1007D00070911101840F951FA61FB71F80930E0102
:1007E00090930F01A0931001B093110188B18C2553
:1007F00088B9F8948501D8011197C8010297F801CA
:1008000040816C91FC0180810E94F6000D5F1F4FBA
:100810000815190581F778948091020190910301E0
:10082000FD2D28E0F202800D911D1124909303010B
:1008300080930201809100019091010138E0F30260
:1008400080199109112490930101809300018091F6
:1008500000019091010144E164E60E9402032B0132
:100860003C01809102019091030144E164E60E9401
:100870000203FE0131967F010EE110E0A301920117
:100880000E9447014EE150E0BE0167587F4FC7010B
:100890000E94DD02F1E0DF1212C08091020190910E
:1008A00003018236924018F0DD24DA944DCF809116
:1008B0000001909101018F359140B0F345CF8FEF4A
:1008C000D81611F0D12C40CF8091020190910301F4
:1008D0008F35914018F4DD24D39436CF80910001F8
:1008E000909101018236924008F42ECFF4CF5058F7
:1008F000BB27AA270E948F040C94D9050E94CB0520
:1009000038F00E94D20520F039F49F3F19F426F404
:100910000C94C8050EF4E095E7FB0C94C205E92F92
:100920000E94EA0558F3BA17620773078407950710
:1009300020F079F4A6F50C940C060EF4E0950B2E3D
:10094000BA2FA02D0B01B90190010C01CA01A00121
:100950001124FF27591B99F0593F50F4503E68F17C
:100960001A16F040A22F232F342F4427585FF3CFBD
:10097000469537952795A795F0405395C9F77EF48E
:100980001F16BA0B620B730B840BBAF09150A1F0D7
:10099000FF0FBB1F661F771F881FC2F70EC0BA0F5D
:1009A000621F731F841F48F4879577956795B795E5
:1009B000F7959E3F08F0B0CF9395880F08F09927E0
:1009C000EE0F9795879508950E94F8040C94D90529
:1009D0000E94D20558F00E94CB0540F029F45F3FF9
:1009E00029F00C94C20551110C940D060C94C80505
:1009F0000E94EA0568F39923B1F3552391F3951BFF
:100A0000550BBB27AA2762177307840738F09F5F2F
:100A10005F4F220F331F441FAA1FA9F335D00E2E9C
:100A20003AF0E0E832D091505040E695001CCAF709
:100A30002BD0FE2F29D0660F771F881FBB1F2617CC
:100A400037074807AB07B0E809F0BB0B802DBF01A3
:100A5000FF2793585F4F3AF09E3F510578F00C9472
:100A6000C2050C940D065F3FE4F3983ED4F38695DF
:100A700077956795B795F7959F5FC9F7880F911D93
:100A80009695879597F90895E1E0660F771F881F7F
:100A9000BB1F621773078407BA0720F0621B730B32
:100AA000840BBA0BEE1F88F7E09508950E94F205BB
:100AB00088F09F5798F0B92F9927B751B0F0E1F01F
:100AC000660F771F881F991F1AF0BA95C9F714C0CF
:100AD000B13091F00E940C06B1E008950C940C0620
:100AE000672F782F8827B85F39F0B93FCCF3869508
:100AF00077956795B395D9F73EF490958095709565
:100B000061957F4F8F4F9F4F0895E89409C097FBE1
:100B10003EF490958095709561957F4F8F4F9F4FD4
:100B20009923A9F0F92F96E9BB279395F695879518
:100B300077956795B795F111F8CFFAF4BB0F11F4DB
:100B400060FF1BC06F5F7F4F8F4F9F4F16C0882382
:100B500011F096E911C0772321F09EE8872F762FB8
:100B600005C0662371F096E8862F70E060E02AF0F9
:100B70009A95660F771F881FDAF7880F96958795E5
:100B800097F9089597F99F6780E870E060E008950D
:100B90009FEF80EC089500240A9416161706180695
:100BA0000906089500240A94121613061406050671
:100BB0000895092E0394000C11F4882352F0BB0F02
:100BC00040F4BF2B11F460FF04C06F5F7F4F8F4F65
:100BD0009F4F089557FD9058440F551F59F05F3FA0
:100BE00071F04795880F97FB991F61F09F3F79F04F
:100BF00087950895121613061406551FF2CF4695D1
:100C0000F1DF08C0161617061806991FF1CF869552
:100C10007105610508940895E894BB276627772736
:100C2000CB0197F908950E9426060C94D9050E94DD
:100C3000CB0538F00E94D20520F0952311F00C94DA
:100C4000C2050C94C80511240C940D060E94EA05F7
:100C500070F3959FC1F3950F50E0551F629FF0010F
:100C6000729FBB27F00DB11D639FAA27F00DB11D28
:100C7000AA1F649F6627B00DA11D661F829F2227B1
:100C8000B00DA11D621F739FB00DA11D621F839F38
:100C9000A00D611D221F749F3327A00D611D231F0E
:100CA000849F600D211D822F762F6A2F11249F575C
:100CB00050409AF0F1F088234AF0EE0FFF1FBB1F5F
:100CC000661F771F881F91505040A9F79E3F51051E
:100CD00080F00C94C2050C940D065F3FE4F3983E3F
:100CE000D4F3869577956795B795F795E7959F5FC8
:100CF000C1F7FE2B880F911D9695879597F908955A
:100D000097FB072E16F4009407D077FD09D00E94B8
:100D10009A0607FC05D03EF4909581959F4F089563
:100D2000709561957F4F0895EE0FFF1F0590F49128
:100D3000E02D0994AA1BBB1B51E107C0AA1FBB1FD2
:100D4000A617B70710F0A61BB70B881F991F5A9557
:100D5000A9F780959095BC01CD010895F894FFCF37
:0A0D6000E001E001012000000000A6
:00000001FF
